:100000000C94BB020C942E210C9402030C9402035A
:100010000C9402030C9402030C9402030C9402034C
:100020000C9402030C9402030C94BE280C949029A7
:100030000C94EE230C9402030C9402030C94020320
:100040000C9402030C9402030C9402030C9402031C
:100050000C9402030C9463240C9402030C9402038A
:100060000C9402030C9402030C9402030C940203FC
:100070000C9402030C9402030C9402030C940203EC
:100080000C9402030C9402030C9402030C940203DC
:100090000C9402030C9402030C9402030C940203CC
:1000A0000C9402030C9402030C940203A005A00517
:1000B000D205D2051F063D065E075E074806DD062F
:1000C000EE06EE064E075E075E075707FE07FE07C1
:1000D000100810080708100810081008FE07FE078F
:1000E0000C08100810080C08FD29242A1C2B242AAF
:1000F0001C2B702A932A1C2BEA2AF92A35421E004F
:100100001F0020002100220001512B0014001A00C2
:100110000800150017003000290004001600070031
:1001200009000A004B4364621D001B000600190011
:1001300005004E00E000E3000000E200E0002A00BD
:100140004C002D42270026002500240023000151E9
:100150002F00130012000C0018001C002E003400A9
:1001600033000F000E000D000B004D4331723800BC
:1001700037003600100011004A004F0052005100B5
:100180005000E6002C00280001003A003B003C0033
:100190003D003E00010001001E021F022F0230023E
:1001A000310201000100200221022F003000350041
:1001B000010001002202230226022702350201006B
:1001C0000100010001000100010001000100000028
:1001D00043004200410040003F0001000000560083
:1001E000610060005F0054000100000057005E00E5
:1001F0005D005C0055000100000058005B005A00E3
:100200005900000001000000580063006200620015
:1002100001000100010001000100010001000100D6
:10022000010000000000ED000000F90000000100E6
:100230000000EF00EE00F000FA00000001000000F6
:1002400000000000000000000000010000000000AD
:1002500000000000F100F2000100010001000100B7
:10026000010001000100010000000000000000008A
:10027000000000000100000000004F00520051008B
:10028000500000000000AE00A800000000000000C8
:100290000100BB00A900AA00BC0000000100010091
:1002A00000003A003B003C003D003E00C65C000000
:1002B000005CCE5CC35CC45CC75C00000000000056
:1002C000000000000000000001000000000000002D
:1002D000000000000000000000000000000000001E
:1002E0000000000000000000430042004100400008
:1002F0003F00C95C000000000000CA5CCB5CC85C29
:1003000000000000000000000000000000000100EC
:1003100000000000000000000000000000000000DD
:1003200000000000000000000000000000010101CA
:1003300001010101010102020202020202020203A2
:100340000303030303030304040404040404050572
:100350000505050606060606070707070708080835
:1003600008090909090A0A0A0B0B0B0C0C0C0D0DE4
:100370000D0E0E0E0F0F0F1010111111121213137C
:100380001414151516161717181819191A1A1B1BF5
:100390001C1D1D1E1E1F2020212222232424252651
:1003A00026272829292A2B2C2D2D2E2F3031323289
:1003B000333435363738393A3B3C3D3E3F40414295
:1003C000434445464748494A4C4D4E4F505153547B
:1003D000555658595A5B5D5E5F616264656668692F
:1003E0006B6C6D6F7072737577787A7B7D7E8082AF
:1003F000838587888A8C8E8F91939596989A9C9EF8
:10040000A0A2A3A5A7A9ABADAFB1B3B5B7BABCBE07
:10041000C0C2C4C6C9CBCDCFD1D4D6D8DBDDDFE2D4
:10042000E4E7E9EBEEF0F3F5F8FAFDFF26035400FC
:100430006800650020005200650064006F007800CD
:1004400020004B006500790062006F0061007200BF
:10045000640000001403460061006C00620061004B
:1004600074006500630068000000040309040902C9
:100470003B00020100A0FA09040000010301010091
:100480000921110100012240000705810308000A2B
:1004900009040100010300000009211101000122EB
:1004A0007B000705820320000A1201000200000001
:1004B00008444D445200010102000105010902A156
:1004C0000185020901A10005091901290815002566
:1004D0000195087501810205010930093115812551
:1004E0007F95027508810609381581257F9501756C
:1004F000088106050C0A38021581257F95017508CB
:100500008106C0C005010980A101850319012AB730
:1005100000150126B700950175108100C0050C0972
:1005200001A101850419012AA002150126A0029546
:100530000175108100C005010906A101050719E038
:1005400029E71500250195087501810295017508B7
:1005500081010507190029FF150026FF0095067582
:100560000881000508190129059505750191029575
:100570000175039101C011241FBECFEFDAE0DEBF89
:10058000CDBF04B603FE27C08091040390910503FC
:10059000A0910603B09107038730904BA740B04B62
:1005A000D1F41092040310920503109206031092E6
:1005B000070314BE84B7877F84BF0FB6F894A8954D
:1005C00080916000886180936000109260000FBE8F
:1005D000E0E0F8E3099511E0A0E0B1E0E0EEF7E536
:1005E00002C005900D92AA3BB107D9F723E0AAEB10
:1005F000B1E001C01D92A430B207E1F70E94AE162F
:100600000C94EE2B0C94000081E0089581E0089595
:100610000C94060308950C940A031F93CF93DF9361
:1006200000D000D01F92CDB7DEB749835A836B83C9
:100630003091BC0189819A81311114C0662359F02F
:10064000222349F00E94A209182F682F89819A81DC
:100650000E944B0903C00E947609182F69817A8194
:10066000812F04C00E94A20969817A810F900F90A6
:100670000F900F900F90DF91CF911F910C9423104A
:10068000FC01262F408151816281738184810C9409
:100690000D0381E00895CF93DF93EC0160E00E94A9
:1006A0004003BE01DF91CF910C940B030E943912DD
:1006B0000E94CE030C9473120C946F1208950E9442
:1006C000EC070E945E032FEF84E39CE02150804002
:1006D0009040E1F700C000000C9489240F931F9311
:1006E000CF93DF938C0161E00E944003EC01B801DD
:1006F0000E940803882309F444C0B801CE010E9477
:10070000DF1E8823F1F1B801CE010E94311F88233A
:10071000C1F1B801CE010E945C20882391F1B8019B
:10072000CE010E94B21D882361F1F80182818823E5
:1007300009F1CB358DE5D807C1F050F4C115FCE5C2
:10074000DF0781F0CF3DDC45A9F40E94370F19C0C7
:10075000CC35EDE5DE0761F0CD35DD4559F40E947D
:10076000C10D08C00E945F030CC00E94CA0D02C0E8
:100770000E94CD0DC801DF91CF911F910F910C9474
:10078000040380E0DF91CF911F910F9108950895A8
:100790000C94C70381E008950C94CA030895CF9385
:1007A000C82F0E94C8038C2F0E94CC03CF910895BC
:1007B000CF93DF93CDB7DEB72B970FB6F894DEBF9C
:1007C0000FBECDBF4F83588769877A878B876111AA
:1007D0000E94F00D9E012F5F3F4F86E0F9011192BC
:1007E0008A95E9F785E0FE013796D90101900D92CF
:1007F0008A95E1F789819A814C815D81452B31F0A1
:100800009F3F31F491E08F3F19F403C091E001C0A4
:1008100090E090FF09C049815A816B817C818D8174
:100820009E810E94F00C05C0C9010E9449038111FC
:10083000F2CF2B960FB6F894DEBF0FBECDBFDF917F
:10084000CF910895FC01808191810E94E40908956F
:10085000CF93882309F4A9C0C82F8238C1F40E941D
:10086000B22281FDA2C069E3809100019091010153
:100870000E944C230E94220E2FEF81EE94E0215023
:1008800080409040E1F700C0000069E319C0833860
:1008900001F50E94B22280FD88C063E580910001CD
:1008A000909101010E944C230E94220E2FEF81EEB5
:1008B00094E0215080409040E1F700C0000063E5E3
:1008C00080910001909101010E944E23CF910C94E0
:1008D000220E8438C1F40E94B22282FD66C067E411
:1008E00080910001909101010E944C230E94220EF0
:1008F0002FEF81EE94E0215080409040E1F700C05E
:10090000000067E4DDCF8CEF8C0F813AF8F48C2F78
:100910000E94E717811149C06C2F809100019091CE
:1009200001010E941623882349F06C2F8091000159
:10093000909101010E944E230E94220E6C2F809103
:100940000001909101010E944C23C0CF80E28C0FE6
:10095000883048F4C77081E001C0880FCA95EAF773
:100960000E94D30DB3CFEBE5EC0FE33040F4F0E0A1
:10097000EF58FE4F808190E0CF910C94DE22E8E5A5
:10098000EC0FE73150F4F0E0EE0FFF1FED5BFE4F90
:1009900080819181CF910C94F422CD3E30F08C2F48
:1009A0000E94B218CF910C948419CF910895882396
:1009B00009F464C0823879F40E94B22281FF5EC0DB
:1009C00069E380910001909101010E944C230E94F3
:1009D000220E69E310C08338B1F40E94B22280FF76
:1009E0004DC063E580910001909101010E944C236C
:1009F0000E94220E63E580910001909101010E9406
:100A00004E230C94220E843879F40E94B22282FF85
:100A100035C067E480910001909101010E944C2350
:100A20000E94220E67E4E7CF9CEF980F913A10F4F2
:100A3000682FE1CF90E2980F983050F4877091E0E2
:100A400001C0990F8A95EAF7892F0E94D90DD9CF55
:100A50009BE5980F933020F480E090E00C94DE2228
:100A600098E5980F973120F480E090E00C94F42200
:100A70008D3E20F00E940D190C94841908951F9347
:100A8000CF93DF93182FEB010E942804209741F0A9
:100A90008FE99FE00197F1F700C000002197F6CFA2
:100AA000812FDF91CF911F910C94D704893319F0D6
:100AB00060E070E002C060E570E00C943F058823C0
:100AC00021F00E94D30D0C94220E0895882321F06A
:100AD0000E94D90D0C94220E0895CF92DF92EF92CE
:100AE000FF920F931F93CF93DF937C01062FC72FA5
:100AF000FC01D281158112951F700E94A80D8823D8
:100B000099F0DD2389F08C2F807F803421F080E202
:100B1000800F883048F082E00E94720E0E94A80D7B
:100B200091E0D82ED92601C0D12CCC2EC2948FE0D2
:100B3000C8228C2D90E0FC01EA5AFF4F0C948A2BBE
:100B40008C2F807FCF70882311F0C295C07FDD236A
:100B500099F0CC2309F48DC180E2800F883010F029
:100B6000011104C08C2F0E94D30D03C08C2F0E9452
:100B7000E30D0E94220E7DC1802F0E94D704CC235A
:100B800009F49CC180E2800F883010F0011104C08C
:100B90008C2F0E94D90D03C08C2F0E94E90D0E945A
:100BA000220E8CC18C2F807FCF70803211F0C295C5
:100BB000C07F002319F00130C9F022C0DD2371F09D
:100BC000112341F0113031F40E94030E8C2B0E944E
:100BD0000B0E74C10E94030E8C2B1DC0112319F043
:100BE000113009F46BC10E94180E25C0DD2321F0DD
:100BF000163008F063C10EC0153008F05FC11BC08D
:100C0000DD2361F0112331F0F701858180FF31C1CF
:100C10008F7085838C2F0E945F0550C1112359F07E
:100C2000093309F037C1FFEF27EE83E0F150204090
:100C30008040E1F72DC18C2F0E9466053FC18C2FAB
:100C400086958695837019F0813061F037C1DD2378
:100C500021F0802F9C2F937002C080E090E00E94D2
:100C6000DE2234C1DD2321F0802F9C2F937002C03F
:100C700080E090E00E94F42229C1802FDD2319F04A
:100C80000E94B21802C00E940D190E9484191EC150
:100C90008C2F837009F045C0D11114C1402F4295AB
:100CA00046954770440F440F602F6F70862F90E079
:100CB000A0E0B0E0042E04C0880F991FAA1FBB1F3C
:100CC0000A94D2F704FF10C00FE010E020E030E0FB
:100CD00004C0000F111F221F331F4A95D2F7009541
:100CE00010952095309503C000E010E09801C6955E
:100CF000C695C370BC01CD01602B712B822B932B49
:100D0000C23049F058F4C13019F00E946108DAC0CD
:100D10000E944F08D7C00E947308D4C00E944D089B
:100D2000D1C0DD2319F08C2F817001C086958823F6
:100D300009F4C8C0402F429546954770440F440FB0
:100D4000602F6F70862F90E0A0E0B0E0042E04C00A
:100D5000880F991FAA1FBB1F0A94D2F704FF10C067
:100D60000FE010E020E030E004C0000F111F221F50
:100D7000331F4A95D2F7009510952095309503C002
:100D800000E010E09801C695C695C370BC01CD0186
:100D9000602B712B822B932BC23049F058F4C13059
:100DA00019F00E9426098EC00E9414098BC00E946F
:100DB000380988C00E94870885C0CF70DD2339F0CC
:100DC0008C2F0E94AD08802F0E945F057BC0802F72
:100DD0000E9466058C2F0E94CE0874C0023F01F16C
:100DE00028F4003F41F0013FA1F03FC0033FF9F07C
:100DF000043F39F13AC0DD2341F0153008F05EC000
:100E00008C2F8F710E94F30859C0163008F056C01D
:100E1000F7CFDD2339F08C2F8F710E94AD084EC0C3
:100E2000DD23C9F38C2F8F710E94CE0847C0DD23CC
:100E300029F08C2F8F710E94980840C00E9493085F
:100E40003DC0DD2349F0CF718C2F0E94AD0863E0D7
:100E50008C2F0E94570E32C081E00E94720E123019
:100E600068F182E00E94720E29C0DD2331F0112367
:100E700091F2802F0E94280421C0112399F2093396
:100E800049F49FEFE7EEF3E09150E040F040E1F7E6
:100E900000C00000802F0E94D70410C04C2F4F705C
:100EA000602FC7010E941F100E94120A0FC04C2F12
:100EB0004F70602FC7010E94221008C088EF8C0D70
:100EC000843020F40E94B2220E94CF03DD20C9F0BA
:100ED0000E94A40D80FD15C0F70112820E949E0D94
:100EE0000E94AD08C7010E94A2070E949E0DDF91DB
:100EF000CF911F910F91FF90EF90DF90CF900C94C6
:100F0000CE08DF91CF911F910F91FF90EF90DF906E
:100F1000CF9008950F931F93CF93DF93EC016881D7
:100F200079818A810E94EF098C010E944A090E94FE
:100F30003B08B801CE010E946D05DF91CF911F9152
:100F40000F910895CF93DF93EC01988189812B81D4
:100F50003C81232B31F08F3F31F481E09F3F19F426
:100F600003C081E001C080E080FD19C0CE010E9475
:100F70006E0381110CC00E94A80D882381F08A8124
:100F8000882369F082E0DF91CF910C94720ECE013C
:100F90000E948A07CE01DF91CF910C944B03DF9121
:100FA000CF91089580E090E00E94DE2280E090E002
:100FB0000E94F4220E94F00D0E94000E0E94220E58
:100FC0000E94B51A0C94841980910001909101013E
:100FD0000E9450230C94D2070E94E00D0C94E40769
:100FE000E92FE295EF704E2F50E0FA013297EE3084
:100FF000F105B0F4EA59FF4F0C948A2B803F91F031
:1010000018F4883E68F40EC0843F51F40BC0883E4B
:1010100048F0813F29F406C093FB882780F90895A2
:1010200080E0089581E00895FC01808191810E9413
:10103000E4090E94F0070895CF93DF9300D000D019
:101040001F92CDB7DEB70F900F900F900F900F90BB
:10105000DF91CF910895CF93DF9300D000D000D0DF
:10106000CDB7DEB726960FB6F894DEBF0FBECDBF64
:10107000DF91CF910895089508950C943C080C9445
:101080003D080E943F086093EE017093EF0180934A
:10109000F0019093F1010C94D2070C9441080F9346
:1010A0001F930091EE011091EF012091F00130911A
:1010B000F101602B712B822B932B1F910F910C94BC
:1010C00041080F931F930091EE011091EF012091C1
:1010D000F0013091F10160237123822393231F914A
:1010E0000F910C9441080F931F930091EE01109102
:1010F000EF012091F0013091F101602771278227E3
:1011000093271F910F910C9441080C943C080E9466
:1011100085086093EA017093EB018093EC01909352
:10112000ED010C94D20760E070E0CB010C948708CD
:101130000F931F9341E050E060E070E08A019B0153
:1011400004C0000F111F221F331F8A95D2F7C90157
:10115000B8011F910F910C9487080F931F9341E0E2
:1011600050E060E070E004C0440F551F661F771F19
:101170008A95D2F78091EA019091EB01A091EC0160
:10118000B091ED018A019B01082B192B2A2B3B2BD7
:10119000C901B8011F910F910C9487080F931F93F9
:1011A00041E050E060E070E004C0440F551F661F4E
:1011B000771F8A95D2F740955095609570958091EC
:1011C000EA019091EB01A091EC01B091ED018A014F
:1011D0009B01082319232A233B23C901B8011F912E
:1011E0000F910C9487080F931F9341E050E060E04B
:1011F00070E004C0440F551F661F771F8A95D2F711
:101200008091EA019091EB01A091EC01B091ED0188
:101210008A019B01082719272A273B27C901B80102
:101220001F910F910C9487080F931F930091EA016F
:101230001091EB012091EC013091ED01602B712BAD
:10124000822B932B1F910F910C9487080F931F9360
:101250000091EA011091EB012091EC013091ED0138
:1012600060237123822393231F910F910C9487088D
:101270000F931F930091EA011091EB012091EC0173
:101280003091ED0160277127822793271F910F91DD
:101290000C948708089527E0929F800D1124E82F71
:1012A000E695E695E695877051E001C0550F8A9561
:1012B000EAF785E0E89FF0011124E354FE4F20E0B7
:1012C00030E070E04081CB01022E02C096958795F8
:1012D0000A94E2F78170819584278523842781937E
:1012E0002F5F3F4F2530310569F7089527E0929F22
:1012F000800D1124682F669566956695982F9770D6
:1013000085E0689FB001112440E050E080E0FB01DF
:10131000E40FF51FE354FE4F208130E0092E02C098
:10132000369527950A94E2F721703327042E01C0E1
:10133000220F0A94EAF7822B4F5F5F4F4530510529
:1013400031F70895BF92CF92DF92EF92FF920F9301
:101350001F93CF93DF938C01C090EA01D090EB01F3
:10136000E090EC01F090ED018091EE019091EF01A1
:10137000A091F001B091F101C82AD92AEA2AFB2AEA
:10138000CFE1D0E0D701C6010C2E04C0B695A795D9
:10139000979587950A94D2F780FD04C0219790F71E
:1013A000B12C07C0BC2EB8018C2F0E945A11019796
:1013B000A9F38B2DDF91CF911F910F91FF90EF90AB
:1013C000DF90CF90BF900895CF93DF93EC010E9400
:1013D000A209BE010E945A11DF91CF9108951F9377
:1013E000CF93DF93EB019091BC01992321F0CB01C6
:1013F0000E94E40913C0882349F0CB010E94A2098E
:10140000182F682FCE010E944B0904C0CB010E9407
:101410007609182FBE01812F0E945A11DF91CF91BA
:101420001F910895EF92FF920F931F93CF93DF9335
:101430008C01892B09F46CC0F12CEE24E394E801B3
:101440002196F8018491843740F4843008F051C02B
:10145000813081F0823019F15BC0853709F444C0D6
:10146000A8F19CE7980F903708F052C08F770E9440
:10147000D70441C00E5F1F4FFE01849190E2980F88
:10148000983050F48770FE2D01C0FF0F8A95EAF75F
:101490008F2F0E94F30D14C00E9428042DC00E5FF0
:1014A0001F4FFE01849190E2980F983060F487708E
:1014B000FE2D01C0FF0F8A95EAF78F2F0E94F90DCC
:1014C0000E94220E19C00E94D70416C00E5F1F4F43
:1014D000FE01C491CC2381F08FE99FE00197F1F7E1
:1014E00000C00000C150F6CF0E5F1F4FFE01F49008
:1014F00003C00E9428048E018F2D882309F49FCFFA
:10150000EFE9FFE03197F1F700C000008150F5CF1F
:10151000DF91CF911F910F91FF90EF9008951F934E
:10152000CF93DF93C091F20116E08091F301C817C9
:1015300099F0D0E01C9FF0011D9FF00D1124EC509C
:10154000FE4F4081518162817381848195810E9427
:101550002B082196C770E9CFDF91CF911F91089595
:101560004091240250912502609126027091270239
:1015700080912802909129020C942B080F931F93BD
:10158000CF93DF938091290282958F7009F05DC01F
:1015900080912602882309F458C08091F2011091AD
:1015A000F3016091240270912502C0912702D0912D
:1015B000280291E06F3F09F090E0292F06E08117A3
:1015C00009F443C0209721F07F3F21F030E003C0B1
:1015D00031E001C0322F90E030FD34C0089FF001AF
:1015E000099FF00D1124DF01AC50BE4F11963C91C4
:1015F0001197371327C03C91361324C012963C91A3
:10160000129731111FC013964D915C9114974C1B8A
:101610005D0B483C5105B0F4809129028F708061C8
:1016200080932902E750FE4F80818F708061808314
:1016300084E292E00E94A207DF91CF911F910F9167
:101640000C948F0A01968770BACFDF91CF911F91CA
:101650000F9108959F92AF92BF92CF92DF92EF9237
:10166000FF920F931F93CF93DF93CDB7DEB76197B0
:101670000FB6F894DEBF0FBECDBF8C0185E0F80138
:10168000DE011D9601900D928A95E1F7F801E28046
:101690009091240260912502209127023091280226
:1016A0002115310531F06F3F31F481E09F3F19F48E
:1016B00003C081E001C080E0F82FF1709F2E80FD13
:1016C0003FC1F80140815181A380B48084E2C82EDB
:1016D00082E0D82EF0902602F501E21BF30BFF20EA
:1016E00009F4D9C080912902E83CF10508F095C0C1
:1016F000282F207F09F052C0561313C0491311C080
:10170000FE2CE1100EC08F708061809329020E9430
:10171000B00AC6010E94A20780912902F8018583C0
:101720004CC1AB2831F05F3F31F481E04F3F19F4F9
:1017300003C081E001C080E080FD03C081E08E2510
:1017400002C080E090E0F82FF170FF2E80FF1CC0F7
:101750008091F2012091F30136E0821709F40BC168
:1017600090E0389FF001399FF00D1124EC50FE4FAE
:101770006181561306C06081461303C06281E61280
:1017800003C001968770E9CFFE2CEE2009F415C145
:101790008091290281608093290254C0561306C0AB
:1017A000491304C0E11002C0F80199C0C8010E94A9
:1017B0001408882361F1EE2051F120912902822F33
:1017C00082958F7090E0029774F08091240290913E
:1017D000250298878F831986BB86AA862C87CE011F
:1017E00007960E94A20786E0F801A4E2B2E0019009
:1017F0000D928A95E1F70E94BE0A0E94B00A0AC0C3
:10180000561711F1C8010E94140881112CC0C8019B
:101810000E94A207FF24F394D0C0282F207F81F7D5
:101820007A2DB98AA88A6E2D89890E941C0884E2C3
:1018300092E00E94A20786E0F60111928A95E9F7EC
:101840000E94B00AF12CB9C04913DCCFE110DACF05
:10185000F8018583C8010E94A20786E0F601119273
:101860008A95E9F7AAC0EE2091F220912902822FF1
:1018700082958F7090E002970CF4B5CF809124028E
:10188000909125029A8389831B82BD82AC822E832C
:10189000CE010196A6CFE83CF10508F044C0FE2C2D
:1018A000EE2009F4B4CF561330C049132EC0209156
:1018B000290220FD21C0822F82958F70482F50E091
:1018C00041155105C9F0F80125834F30510541F00C
:1018D0008F5F982F9295907F822F8F70892B8583B1
:1018E000C8010E94A20786E0F801A4E2B2E00190DC
:1018F0000D928A95E1F73CC086E0F801A4E2B2E0DF
:1019000001900D928A95E1F758C0C8010E94140811
:10191000811169CF80912902816080932902C801D9
:101920000E94A2074AC07A2DB98AA88A6E2D898999
:101930000E941C0886E0F60111928A95E9F718C00A
:10194000EE2009F464CFC8010E941408F82E882301
:1019500009F45DCF86E0F801A4E2B2E001900D92B7
:101960008A95E1F784E292E00E9422040E94BE0A76
:101970000E94B00A22C04D875E878D859E850E9499
:10198000E409292F22952F70223028F49F7039F016
:10199000811105C00BC0243028F49F7049F4805E8B
:1019A000883020F0C8010E94A2079F2CF92C05C0A6
:1019B000F8019581907F99F7F9CF8F2D61960FB639
:1019C000F894DEBF0FBECDBFDF91CF911F910F9175
:1019D000FF90EF90DF90CF90BF90AF909F900895D1
:1019E0001F93CF93DF93CDB7DEB72C970FB6F89444
:1019F000DEBF0FBECDBF4F83588769877A878B873D
:101A00009C87CE0107960E942A0B8823D1F09F81E4
:101A100088852A853B85232B31F08F3F31F481E087
:101A20009F3F19F403C081E001C080E080FD47C002
:101A30004F81588569857A858B859C850E942B0806
:101A40003EC086E0FE013796DE01119601900D92B0
:101A50008A95E1F7FF81E8856A857B8561157105C7
:101A600031F0EF3F31F481E0FF3F19F403C081E032
:101A700001C080E080FD23C02091F30130E0C90166
:101A80000196877099274091F20150E084179507DD
:101A9000F1F1F983EA837D836C8396E0929FD00114
:101AA000939FB00D1124AC50BE4FFE0131960190B2
:101AB0000D929A95E1F78093F3010E948F0A16E048
:101AC0008091F2019091F301891771F1189FC00183
:101AD00011248C509E4F0E942A0B882329F1E091FB
:101AE000F2011E9FF0011124EC50FE4F4081518104
:101AF00062817381848195810E942B088091F2011B
:101B000090E00196877099278093F201D9CF0E94C7
:101B1000EC071092F3011092F201E4E2F2E086E0A9
:101B2000DF011D928A95E9F72C960FB6F894DEBF77
:101B30000FBECDBFDF91CF911F91089580912A02F2
:101B4000859585958595089580912A0287700895D9
:101B500090912A02977081E009F480E008959091B5
:101B6000A80292FB222720F9281751F080FB92F956
:101B70009093A8028091A7029091A8020C94B30EB2
:101B800008958091A80282FB882780F991E0892737
:101B90000C94AF0D81E00C94AF0D80E00C94AF0D70
:101BA00080913602089590913602892B80933602F7
:101BB0000895809590913602892380933602089586
:101BC00010923602089590913502892B8093350248
:101BD0000895809590913502892380933502089568
:101BE00010923502089590913402892B809334022B
:101BF000089580959091340289238093340208954A
:101C000010923402089580912B02089508950C9447
:101C1000060E0C94070E9091A80292FD08C09091B8
:101C20002B02981721F080932B020C94090E089533
:101C300080912B02882329F010922B0280E00C94D3
:101C4000090E0895E0910001F091010180913602A2
:101C50008083E0910001F091010190818091350233
:101C6000892B8083E0910001F091010190818091A6
:101C70003402892B808380912B02882381F0E091AC
:101C80000001F09101019081892B808380910001F6
:101C9000909101010E940A2381110E94180E8091E7
:101CA0000001909101010C94C5220C94060E9091B4
:101CB000A80292FD10C098E0899F90011124262B64
:101CC00020932A020E94AD0880912A02859585956D
:101CD00085950C94550E0C94AD0810922A0280E064
:101CE0000C94550E20912A028095822380932A021B
:101CF000982F977041F430E0482F082E000C550BB8
:101D00002417350721F49091A80292FF07C085950A
:101D1000859585950E94CE080C946D0E089580E0FF
:101D200090E00E94B42B21E0893E9E4F09F020E014
:101D3000822F089582E090E00C94A62B83E090E03F
:101D40000C94A62BCF9384E090E00E94A62BC82F82
:101D500082E290E00E94A62B2C2F30E0A901582BA4
:101D6000CA01CF910895CF93C92F682F84E090E0E6
:101D70000E94BA2B6C2F82E290E0CF910C94BA2B88
:101D8000AB01BC018FE090E00C94CC2BAB01BC010B
:101D900083E190E00C94CC2B60E070E0CB010C94DC
:101DA000C60E60E070E0CB010E94C00E0C94CC0E19
:101DB00069EE7EEF80E090E00E94D82B60E082E048
:101DC00090E00E94BA2B60E083E090E00E94BA2B82
:101DD0001092EE011092EF011092F0011092F101B9
:101DE00060E084E090E00E94BA2B60E082E290E044
:101DF0000E94BA2B60E085E090E00E94BA2B60E080
:101E000086E090E00E94BA2B6FEF87E090E00E949E
:101E1000BA2B40E050E0BA0188E090E00E94CC2B61
:101E200060E08DE090E00E94BA2B40E050E0BA0103
:101E300088E190E00E94CC2B60E087E190E00E9476
:101E4000BA2B40E050E0BA018CE190E00E94CC2B2C
:101E500060E070E080E290E00E94D82B40E050E02B
:101E6000BA0188E190E00E94CC2B0C94D10E0C9426
:101E7000D80E682F8EE090E00C94BA2B0E942C2490
:101E80006093460270934702809348029093490200
:101E90006093420270934302809344029093450200
:101EA000089585B7806885BF85B7806885BF089528
:101EB0000C941E1408950C945A0F0C945A0F0C9401
:101EC0005D0F0C945A0F0C94610F0C945A0F0E94E2
:101ED000510F86E392E10E949A240E94650F0C94B0
:101EE000630F0E945B0F0C945A0F0E9417240E94EC
:101EF00057230E9419130E94541E0E94391D0C94EE
:101F00005F0F9F92AF92BF92CF92DF92EF92FF92BC
:101F10000F931F93CF93DF93CDB7DEB72A970FB6FA
:101F2000F894DEBF0FBECDBF0E94931381110E94B3
:101F30003E0F88E3A82E82E0B82E00E010E0902E3D
:101F4000802F0E945D12D82EF501C1905F01C82636
:101F5000B1F40F5F1F4F0A30110589F78FEF8983A6
:101F60008A831B820E9420248160782F9D838C832A
:101F700049815A816B818D810E94D8032FC0809145
:101F80004A0281FD0E946312E12CFF24F3948C2D00
:101F90008F21F1F00E94580F882399F0EE829F82E2
:101FA000DF2081E009F480E088870E94202481609E
:101FB000782F9A8789874E815F8168858A850E94FC
:101FC000D803F801E85CFD4F8081F826F08206C056
:101FD000E394FF0CF7E0EF12DACFBBCF0E94A21917
:101FE0000E94B222909137028917B9F00E94B22262
:101FF000809337022A960FB6F894DEBF0FBECDBF8E
:10200000DF91CF911F910F91FF90EF90DF90CF90D4
:10201000BF90AF909F900C94CF032A960FB6F89480
:10202000DEBF0FBECDBFDF91CF911F910F91FF900B
:10203000EF90DF90CF90BF90AF909F90089580E099
:1020400090E00895089526E4829FC0011124FC01C8
:1020500027E0729FE00DF11D1124E60FF11DEE0F38
:10206000FF1FE450FF4F859194910895880F991FA9
:10207000FC01E45DFC4F859194910895CF93DF932B
:102080000E945F11EC01811520E5920708F03FC026
:10209000811540E4940708F0D2C0883E910500F510
:1020A000803E910508F002C1883A910570F4853AA6
:1020B000910508F0A6C08130910509F49FC008F48D
:1020C000F2C0049708F0F2C0EEC08F3B910508F40F
:1020D000A1C0803C910508F4E6C0805C9109A5C0D0
:1020E000811550E2950760F4C11581E0D80708F02A
:1020F000DDC0CD3ED10508F4D6C0CE019065D7C075
:10210000811520E3920708F093C09F708EC081155F
:1021100045E5940708F046C0811554E5950708F099
:10212000A6C0C11582E5D80718F5C11521E5D2076B
:1021300008F088C0CE01F4E096958795FA95E1F70E
:10214000282F23703C2F337081E090E002C0880F6D
:10215000991F3A95E2F79C68922B2C2F2F702695A9
:10216000269540E2249F90011124822B932B9FC03F
:102170009E01237033279C2F96959695C115D345C4
:1021800008F065C041E050E002C0440F551F2A9599
:10219000E2F780E2989F90011124CA01822B932BD1
:1021A0009C6885C0811559E5950798F4C11588E5A7
:1021B000D80708F061C0C11526E5D20708F073C042
:1021C0008C2F0E94F3118F7190E0982F88279062D6
:1021D0006EC081154AE5940708F453C090568115E6
:1021E000904208F060C08D2F8F710E94F3119E0104
:1021F000332730628F71A901582B53C081E090E0E2
:1022000056C0855AC82FD0E0CE55DE4F888190E069
:1022100090644DC0885AC82FD0E0CC0FDD1FCC5839
:10222000DE4F88819981946442C00E9436103FC07D
:102230009927D3FF02C0986C3AC0906C38C09F7049
:10224000906A35C09C2F8827816F906A30C041E02A
:1022500050E002C0440F551F2A95E2F780E2989F94
:1022600090011124CA01822B932B9A6820C0982FC9
:102270008827846F906A1BC09C2F8827806F906A84
:1022800016C08F700E94F3119E0194E03695279539
:102290009A95E1F72F7030E0322F22273069A9019B
:1022A000482BCA0104C080E090E001C0CE01DF915C
:1022B000CF9108950E9423100E943E100895823805
:1022C000910569F1B0F48133910509F46DC048F4CA
:1022D0008932910509F463C08A32910509F469C015
:1022E00008958533910509F455C089339105B9F0F6
:1022F0000895833E910569F138F4803E9105B1F06F
:10230000823E910509F10895863E9105A9F1873E27
:102310009105B9F1843E910509F064C023C0209174
:10232000A70220FD4FC021FD4DC008958091A70256
:1023300080FD44C08091A80280FF44C08091A70224
:1023400084FD42C083EE4DC08091A70282FF38C059
:10235000F5CF8091A70282FD33C08091A80280FD55
:1023600031C0ECCF8091A80281FF32C08091A702DA
:1023700084FD2AC087EE35C08091A70283FF26C066
:10238000F5CF8091A70283FD21C08091A80281FD35
:102390001FC0ECCF8091A70285FD1CC01DC080919D
:1023A000A70285FD19C016C08091A70286FD16C040
:1023B00017C08091A70286FD13C010C089E311C029
:1023C00082EE0FC080EE0DC080E00BC086EE09C02B
:1023D00084EE07C089E205C085E303C08AE201C03C
:1023E00081E390E008959091A70292FF0DC0282FFD
:1023F0002871283019F4877F846006C0282F247143
:10240000243011F48B7F886093FF0DC0282F287132
:10241000283119F4877E846106C0282F2471243165
:1024200011F48B7E88612091A80220FF0DC0382F07
:102430003871383019F4877F816006C0382F3171C8
:10244000313011F48E7F886021FF0DC0282F287154
:10245000283119F4877E816106C0282F217121312E
:1024600011F48E7E886194FD877E089580E0089542
:1024700008950E948F0E811102C00E94370F0E94A2
:102480009A0E80934A020E94A20E9093A802809313
:10249000A7020E9438120E949E0E682F70E080E012
:1024A00090E00E944D086091EA017091EB018091EB
:1024B000EC019091ED010C948508E82FF0E0ED54CB
:1024C000FD4F80810895089580EA8A95F1F7089577
:1024D00000C008950C94641208950C946C120C942E
:1024E0006D120C946C120C947112F894E82FE29512
:1024F000EF70F0E031A1282F2F7081E090E001C053
:10250000880F2A95EAF7982F9095932391A392A18B
:10251000892B82A37894089508950C948C120F93BC
:102520001F93CF93DF93CCEAD1E089918F3F11F0D5
:102530000E94751281E0C13BD807B9F7C5EAD1E026
:102540000CEA11E089918F3F11F00E9475120C176F
:102550001D07C1F7DF91CF911F910F910895CF9281
:10256000DF92EF92FF920F931F93CF93DF938C0133
:10257000C62FD0E0CE0184559E4F7C01FC01908196
:102580009F3F09F44DC0D62EF894E92FE295EF70E5
:10259000F0E081A19F7021E030E001C0220F9A9508
:1025A000EAF7822B81A382A12095282322A3789485
:1025B0000E946812E5EAF1E020E030E0C12C51E031
:1025C00041914F3FB1F0A42FA295AF70B0E090962B
:1025D0008C9190E04F7002C0959587954A95E2F7EF
:1025E00080FD07C0852F022E01C0880F0A94EAF7EC
:1025F00001C080E0C82A2F5F3F4F2730310501F727
:10260000F70180818F3F11F00E94751261E0C110C7
:1026100001C060E08D2D0E946A12C00FD11FC882D8
:10262000DF91CF911F910F91FF90EF90DF90CF90AE
:1026300008950E9438148091020180910201811155
:1026400002C095E001C090E09093BE0285E0891B36
:102650008093BD020E948F12E9EAF2E0A3EBB2E0A0
:1026600011921D9282E0E33BF807D1F785E00E94CA
:10267000E7130E9456030C9442140F931F93CF93B9
:10268000DF9300D000D01F92CDB7DEB70E941E149A
:102690006091BE02882379F18E010F5F1F4F85E0A4
:1026A000F80111928A95E9F7862F90E0B8018D54D0
:1026B0009D4F0E945014E091BD029E012A5F3F4F42
:1026C000F0E0ED54FD4FD801882361F010E08D91CA
:1026D0009081981711F0808311E03196A217B3070B
:1026E000B1F706C011921D92A217B307D9F711E0F6
:1026F0000E945C030DC070E06D547D4F8091BD025F
:1027000090E08D549D4F0E94E0140E948D1210E0C5
:10271000812F0F900F900F900F900F90DF91CF911E
:102720001F910F910895EF92FF920F931F93CF93F4
:10273000DF93CDB7DEB72A970FB6F894DEBF0FBE92
:10274000CDBF8E010F5F1F4F8AE0F80111928A956D
:10275000E9F7F12C6F2DC8010E94AF12F394F5E058
:10276000FF12F8CF4AE050E0B80189EA92E00E94F7
:10277000902B7C0121E0892B09F420E0E114F10485
:1027800041F08AE0F801A9EAB2E001900D928A9541
:10279000E1F76091BE0270E06D547D4F45E089EA3B
:1027A00092E00E94E813EF2819F40E943D1302C042
:1027B00081E090E02A960FB6F894DEBF0FBECDBF41
:1027C000DF91CF911F910F91FF90EF9008950895A1
:1027D000FF920F931F93CF93DF938C01F62ED72F89
:1027E000C42F222349F081E080934D020E942024CF
:1027F00090934C0280934B0280914D028823C1F04C
:1028000080914B0290914C020E943824059780F0F1
:10281000EF2DFD2FD8014C2F50E0CD01801B910BE7
:10282000841795071CF48D918193F7CF10924D0278
:10283000DF91CF911F910F91FF90089580915002E9
:1028400081110DC00E94552B811102C082E001C090
:1028500081E080935002823011F40E94502B81E07D
:1028600090915002913009F080E008950C941E146C
:102870000E943614809302010E941E1481110C9450
:10288000881408950E941E14811102C00C948A14A9
:10289000089581E0909151029A3008F080E0089507
:1028A0000F931F93CF93DF93EC018B018091510223
:1028B0008A3038F4B801CE010E94DE1481111DC0A7
:1028C0000AC080914E0290914F020E943824843FAA
:1028D000914080F715C0809151028F3F19F08F5FB2
:1028E00080935102809151028A3060F00E9420242E
:1028F00090934F0280934E0203C01092510202C087
:1029000080E001C081E0DF91CF911F910F91089588
:102910000C94E8200C94EB20EF92FF920F931F93FE
:10292000CF93DF937901C82F880FDD0B4115510537
:10293000A9F08AE08C9FF0018D9FF00D1124ED5FCE
:10294000FE4F838194818E5A9D4F228130E0421741
:10295000530708F49A01A9010E949D2BCE010E9401
:10296000F521892B09F50115110501F18AE08C9FEC
:10297000F0018D9FF00D1124ED5FFE4F458150E079
:102980000417150708F4A8018AE08C9FF0018D9FB9
:10299000F00D1124ED5FFE4F668177816E5A7D4FF9
:1029A000C7010E949D2B02C080E001C081E0DF9141
:1029B000CF911F910F91FF90EF9008950C944516C1
:1029C0000C9469160F931F93CF93DF9300D000D020
:1029D000CDB7DEB76091710270917202809173027F
:1029E000909174020E944724643671058105910517
:1029F00028F10E947D23DC01CB010296A11DB11DAF
:102A000089839A83AB83BC8300E010E020E030E050
:102A100044E050E0BE016F5F7F4F82E00E948C1463
:102A2000182F882361F00E942C2460937102709308
:102A30007202809373029093740201C011E0812F9F
:102A40000F900F900F900F90DF91CF911F910F91EA
:102A50000895AF92BF92CF92DF92EF92FF920F93C1
:102A60001F93CF93DF937C015B016A010E9449149D
:102A7000811103C001E010E002C00AE010E0C1E0F3
:102A8000D0E0F894B501C701F60109957894811159
:102A900015C021960C171D0794F0CC9F9001CD9F77
:102AA000300D300D112480E090E045E34A95F1F7B8
:102AB0000000019682179307C1F7E3CF81E0DF9111
:102AC000CF911F910F91FF90EF90DF90CF90BF902B
:102AD000AF9008950F931F93CF93DF93CDB7DEB7D9
:102AE00028970FB6F894DEBF0FBECDBFCE0101967A
:102AF0000E94721D18856091750270917602809116
:102B00007702909178020E9447246436710581050E
:102B1000910510F41123D9F000E010E020E030E03E
:102B200048E050E0BE016F5F7F4F83E00E948C144D
:102B3000882359F00E942C246093750270937602CA
:102B4000809377029093780202C080E003C00E94D5
:102B50006F1D81E028960FB6F894DEBF0FBECDBF83
:102B6000DF91CF911F910F910895AF92BF92CF92B5
:102B7000DF92EF92FF920F931F93CF93DF9300D0DA
:102B800000D000D0CDB7DEB77B01C090B601D090A9
:102B9000B70101E010E09E012A5F3F4F40E050E0A6
:102BA00060E070E080E00E948C14182F882309F404
:102BB0003EC056018FEFA81AB80A60916D0270915D
:102BC0006E0280916F02909170020E9447246436D9
:102BD00071058105910518F105E010E09E012F5F58
:102BE0003F4F40E050E060E070E081E00E948C14D4
:102BF000182F65E070E0C5010E94551E91E02E81FE
:102C0000281390E0192339F10E942C2460936D025F
:102C100070936E0280936F029093700211C065E012
:102C200070E0C5010E94551E9E818913D5CF85E0B5
:102C3000F6013196DE01119601900D928A95E1F729
:102C4000112349F085E0FE013196A8E6B2E001903B
:102C50000D928A95E1F785E0E8E6F2E0D701019070
:102C60000D928A95E1F7812F26960FB6F894DEBF74
:102C70000FBECDBFDF91CF911F910F91FF90EF90CD
:102C8000DF90CF90BF90AF9008950F931F93CF9395
:102C9000DF93EC018B0145EB55E10E942915882358
:102CA00091F042EE54E1B801CE010E94291588232B
:102CB00051F04AE655E1B801CE01DF91CF911F9165
:102CC0000F910C94291580E0DF91CF911F910F9106
:102CD00008950F931F93CF93DF93F894C091B6019B
:102CE000D091B701CE01019625E0FB01DC010190F6
:102CF0000D922A95E1F765E070E00E94551E8883E9
:102D00007894F8946E817F8188859985009164021A
:102D10001091650220916602309167026017710779
:102D20008207930751F06093640270936502809369
:102D30006602909367020E9460237894F8948989D0
:102D4000882331F060E0CE010A960E94851D198A21
:102D50007894DF91CF911F910F9108950E9498234D
:102D60000E94FB250E9414260E9426260E94710FB5
:102D7000FBCF893289F1F0F4843171F1B0F48730FE
:102D800009F077C08EE18093320182E380933101B4
:102D90008AE08093300184E180932F0188E0809362
:102DA0002C0188E280932B0164C092EE980F9A3038
:102DB000F0F05FC0803509F444C028F48F3409F086
:102DC00058C08AE03FC0813529F0823509F051C0F2
:102DD00081E038C08FEF36C080917B02882379F183
:102DE00010927B0210927A021092790242C08D51A9
:102DF00080937B02833099F038F4813069F082301F
:102E0000D9F481E391E00DC0853099F078F08630F7
:102E100099F48BE291E005C082E391E002C080E387
:102E200091E090937A028093790223C08FE291E03F
:102E3000F8CF8CE291E0F5CF10927B021AC080E0CF
:102E4000089586EFE0917902F0917A02309789F047
:102E50002081082E000C990B820F911D8F3F910548
:102E600019F014F08FEF04C097FF02C0108201C068
:102E7000808381E008950F931F9341E050E060E06C
:102E800070E08A019B0104C0000F111F221F331F35
:102E90008A95D2F7C901B8010E944D081F910F9180
:102EA0000C94EC078B3109F468C058F58B3009F4A9
:102EB00086C078F4863009F445C020F4853009F4E2
:102EC0004BC07FC0873009F44AC0883009F477C00E
:102ED00078C0803109F464C068F48E3009F071C0A4
:102EE00080914A0282FB222720F991E0922790FBF1
:102EF00082F94CC0863109F462C0893109F45FC09F
:102F000060C08A32E1F060F4873209F455C028F4D9
:102F10008E3108F456C08D5150C08932E9F051C04D
:102F2000833450F48A3308F045C0853309F444C033
:102F3000883309F444C045C08334F1F142C00E9493
:102F4000370F3DC080914A02817F8E7F80934A0275
:102F500081E080937C0208950E945F0330C08091DD
:102F60004A02982F9095917090FB80F980934A02C5
:102F7000911125C0897F877F10C080914A0281FB13
:102F8000222720F991E0922790FB81F980934A0251
:102F90009923A9F080914A02816080934A020FC070
:102FA00080914A0283FB222720F991E0922790FB2F
:102FB00083F9ECCF895301C080E00E943B1781E088
:102FC000089580E0089580E008950C94E317CF936E
:102FD000C82F80917C02813069F038F08230C1F5D1
:102FE0008C2F0E94B91681E039C00E94D00D823228
:102FF00089F504C00E94D00D823261F48C2F0E94AA
:10300000E517811104C08C2F0E9452171FC081E068
:1030100090E01CC08C2F0E94E317811116C0C431B0
:1030200089F058F4CB3089F0C031B1F482E080935C
:103030007C0288E30E94B91608C0C93219F0C8336F
:1030400021F00AC010927C0207C081E0817006C0A6
:1030500010927C0280E002C080E0F8CFCF9108950A
:103060008091830280FF0BC06091300185E0689FF2
:10307000B001112475956795759567952BC081FFF3
:1030800009C06091300185E0689FB00111247595F9
:10309000679520C082FF07C06091300185E0689F7E
:1030A000B001112417C0909182029923D1F0609150
:1030B0002F01961788F72091300185E0289F900115
:1030C0001124929FA001939F500D112470E0CA011A
:1030D0000E94762B6038710540F46115710519F472
:1030E00006C065E070E0862F08958FE7089581E0BF
:1030F00008958091830280FF08C060912C0170E0E8
:10310000759567957595679521C081FF06C060919B
:103110002C0170E07595679519C082FF04C060911D
:103120002C0170E010C090918102992399F0609178
:103130002B019617A0F780912C01899FC0011124C3
:1031400070E00E94762B6038710540F461157105BE
:1031500019F406C061E070E0862F08958FE70895A6
:1031600081E008958D3E21F40E943018819504C0BD
:103170008E3E29F40E9430188093870208958F3E76
:1031800021F40E943018819504C0803F29F40E94E8
:103190003018809386020895893F19F40E947918A7
:1031A00005C08A3F31F40E94791881958093880286
:1031B00008958B3F21F40E947918819504C08C3FBB
:1031C00029F40E9479188093890208959FE0980F4E
:1031D000983078F421E030E0A90102C0440F551F77
:1031E0009A95E2F7CA0190918502892B8093850216
:1031F00008958D3F21F48091830281600BC08E3F42
:1032000021F480918302826005C08F3F29F4809170
:10321000830284608093830208958D3E39F49091F7
:10322000870297FF35C01092870259C08E3E29F45D
:10323000909187021916BCF32BC0909186028F3EA5
:1032400029F497FF25C01092860249C0803F19F4E7
:103250001916CCF31DC090918802893F29F41916E4
:10326000BCF4109288023BC08A3F19F497FF10C04B
:10327000F8CF8B3F39F49091890297FF09C01092E3
:1032800089022DC08C3F21F4909189021916BCF35C
:103290009FE0980F983080F421E030E0A90102C04F
:1032A000440F551F9A95E2F7CA01809590918502C7
:1032B00089238093850213C08D3F21F4809183027E
:1032C0008E7F0BC08E3F21F4809183028D7F05C0DD
:1032D0008F3F29F4809183028B7F809383028091BA
:1032E0008602811106C080918702811102C010926E
:1032F000820280918802811106C080918902811129
:1033000002C01092810208950E942024209186021A
:10331000211104C020918702222321F09093800282
:1033200080937F0220918802211104C0209189029C
:10333000222321F090937E0280937D0284E892E024
:103340000C94D022EF92FF920F931F93CF93DF93B1
:1033500000D000D000D0CDB7DEB786E0E4E8F2E0E0
:10336000DE01119601900D928A95E1F7E0908602B8
:10337000F0908702009188021091890210928602D3
:10338000109287021092880210928902E11003C005
:10339000FF2009F45DC080917F02909180020E941D
:1033A0003824AC0190918202992339F020913101A7
:1033B00030E02417350758F04BC0209132018AE0E5
:1033C000289F900111242417350718F041C09F3F12
:1033D00019F09F5F90938202EE2061F00E943018F6
:1033E0001E1414F09FEF01C091E0989F902D1124BE
:1033F00090938602FF2061F00E9430181F1414F091
:103400009FEF01C091E0989F902D11249093870227
:10341000309186023323E1F0209187022223C1F00C
:1034200045EB3403C0011124992319F090938602CF
:1034300003C081E08093860235EB2303C001112491
:10344000992319F09093870203C081E0809387024B
:10345000011103C0112309F45DC080917D02909198
:103460007E020E943824AC0190918102992339F0A8
:1034700020912D0130E02417350758F04BC02091E2
:103480002E018AE0289F900111242417350718F097
:1034900041C09F3F19F09F5F90938102002361F02C
:1034A0000E947918101614F09FEF01C091E0989FC8
:1034B000902D112490938802112361F00E947918B5
:1034C000111614F09FEF01C091E0989F902D1124E8
:1034D00090938902309188023323E1F02091890290
:1034E0002223C1F045EB3403C0011124992319F0C4
:1034F0009093880203C081E08093880235EB230318
:10350000C0011124992319F09093890203C081E02E
:10351000809389028091860281110BC0809187027D
:10352000811107C080918802811103C080918902B6
:1035300081110E948419EB82FC820D831E8386E038
:10354000FE013196A4E8B2E001900D928A95E1F770
:1035500026960FB6F894DEBF0FBECDBFDF91CF9198
:103560001F910F91FF90EF900895E4E8F2E086E05C
:10357000DF011D928A95E9F7109282021092810272
:10358000109283020895EF92FF920F931F93CF93AF
:10359000DF938B01682F11110AC0442329F0E82F13
:1035A000F0E0E45DFC4F6491762F862F75C0212FEB
:1035B00030E0E82FF0E0442321F0E45DFC4FE4919B
:1035C000F0E046E0049FC0011124CFEFD0E0BE013F
:1035D0000E94622B4BEA4603C001479F900D1124C5
:1035E000800F911D800F911D982F990F890FAE01AB
:1035F000421B530B4E9FD0014F9FB00D5E9FB00DED
:1036000011249B2F189FA0011124452F55278E01AF
:10361000041B150B0E9FA0010F9F500D1E9F500DF8
:1036200011247E01E81AF108E29E8001E39E100D4C
:10363000F29E100D1124212F3327C21BD30BCE9FD6
:103640009001CF9F300DDE9F300D11246230710547
:10365000A9F048F46115710569F061307105C9F48C
:103660008B2F752F0DC06430710581F058F06630D6
:10367000710579F47E2F8B2F932F0DC0832F7B2F15
:103680009E2F09C08E2F7B2F952F05C08E2F732F55
:1036900002C07E2F852F692FDF91CF911F910F914F
:1036A000FF90EF90089541E00E94C31A08950E9490
:1036B000531B0895CF93DF93762FE901682F842F52
:1036C0000E94571B798368838A83DF91CF91089585
:1036D0008091C002982F9695913021F08170826080
:1036E0008093C002089588E090E00C94AE2BCF92B6
:1036F000DF92EF92FF926B017C010E94681BB70181
:10370000A60188E090E0FF90EF90DF90CF900C94BE
:10371000CC2BE0ECF2E083E0808311828FEF828398
:1037200083831482ABE8B2E012968C911297836087
:1037300012968C9360817181828193810C94771BA6
:103740009091C402933018F49F5F9093C402882331
:1037500051F06091C0027091C1028091C2029091BB
:10376000C3020C94771B089581E00C94A01B9091E8
:10377000C402992319F091509093C402882351F008
:103780006091C0027091C1028091C2029091C30207
:103790000C94771B089581E00C94B71B70E00C9497
:1037A000291E609134018091C00280FF0AC080917F
:1037B000330123E0829FC00111248B539D4F0C9451
:1037C000CE1B8091350190913601891780F7E82F43
:1037D000F0E09F01220F331FE20FF31FEB53FD4F69
:1037E0001182108212828F5FF0CFE0ECF2E08081D4
:1037F0008E7F808360817181828193810E94771B9B
:10380000EBE8F2E08281816082832FEF80E792E033
:10381000215080409040E1F700C000000C94D11B83
:10382000E0ECF2E080818E7F8083EBE8F2E0828141
:10383000816082832FEF80E792E0215080409040AA
:10384000E1F700C000000C94D11B9091C00290FFE2
:1038500016C09091350120913601921770F4E92F2E
:10386000F0E0DF01AA0FBB1FEA0FFB1FEB53FD4F78
:103870008183608342839F5FF0CF0C94D11B0895B6
:10388000EF92FF920F931F93CF93DF9300D01F927D
:10389000CDB7DEB79091C00290FF3DC0E22E142F4D
:1038A000062FF82EE92FE695F0E0E854FE4F8081D0
:1038B00080938B029E7F923059F49E012F5F3F4F81
:1038C0008F2D0E945A1B4B8169818A810E94251C81
:1038D0008091C102F81208C08091C202081304C08E
:1038E0008091C302181729F080918D028260809325
:1038F0008D02F092C1020093C2021093C302EE2027
:1039000051F06091C0027091C1028091C202909109
:10391000C3020E94771B0F900F900F90DF91CF9101
:103920001F910F91FF90EF900895E0ECF2E09181EC
:10393000282F4381628188E0890F0C94401C81E02C
:103940000C94951CE0ECF2E09181282F4381628178
:1039500088EF890F0C94401C81E00C94A21CE0ECD1
:10396000F2E0628121E1620F08F46FEF282F4381BA
:1039700081810C94401C81E00C94AF1CE0ECF2E0DF
:10398000628121E1621B08F460E0282F438181817C
:103990000C94401C81E00C94BE1CE0ECF2E04381EE
:1039A00021E1420F08F44FEF282F628181810C94AE
:1039B000401C81E00C94CD1CE0ECF2E0438121E15D
:1039C000421B08F440E0282F628181810C94401C46
:1039D00081E00C94DC1C20E00C94401C8091C0021F
:1039E00080FF1DC0817082608093C00280918D0233
:1039F000816080938D02662351F06091C0027091C6
:103A0000C1028091C2029091C3020E94771B409133
:103A1000C3026091C2028091C1020C94EB1C089514
:103A2000682F81E00C94EE1C81E00C94101D682F2F
:103A30009091C00296958FEF890F09F481E00C9464
:103A4000EE1C81E00C94171D61E00C94EE1CE0EC80
:103A5000F2E080818160808386950C94241D8091A2
:103A6000C00280FD0C94F51B0C94271D60E00C94A3
:103A7000EE1C80918A02811131C00E948F0E81114B
:103A800004C00E94370F0E94891B0E94731B609321
:103A9000C0027093C1028093C2029093C3028091CE
:103AA0008D02836080938D026E7F61F40E94891B7A
:103AB0000E94731B6093C0027093C1028093C20284
:103AC0009093C3020E94681B8091C00280FF03C0D4
:103AD00086950E94361D81E080938A020895109297
:103AE0008D02089525E0E0ECF2E0DC0101900D92FA
:103AF0002A95E1F720918B0230918C0240918D0242
:103B0000FC0125833683478308951F93CF93DF936A
:103B1000EC01162F8F8180FF0FC0888180FF0AC0C3
:103B20008091C00281608093C002888186950E9446
:103B3000EE1C02C00E94101C8F8181FF09C0212F42
:103B40004B816A818981DF91CF911F910C94401C38
:103B5000DF91CF911F910895882311F0FA0101C0E0
:103B6000FB0109941F93CF93DF93FB011281111185
:103B70006BC0EC010E94D00D8272CA3CFCE5DF07ED
:103B800009F450C0C0F4C63CECE5DE07E1F148F4AE
:103B9000C43C9CE5D90759F178F5C33CDC4521F1DB
:103BA00021C0C83C9CE5D90799F1B8F54FE95CE123
:103BB0006CEA7CE125C0CE3CFCE5DF0709F441C09E
:103BC00050F4CC3CECE5DE0791F1B0F549ED5CE159
:103BD00068EE7CE115C0C73D8CE5D807A8F1CE356D
:103BE000DD4591F111E030C00E942F1D2DC041E252
:103BF0005DE164E17DE104C044E15DE161E27DE11C
:103C00000E94AC1D21C04CEA5CE16FE97CE1F8CF79
:103C10004AEC5CE16BEB7CE1F3CF4BEB5CE16AECF3
:103C20007CE1EECF48EE5CE169ED7CE1E9CF4BEC65
:103C30005BE164EB7BE1E4CF44EB5BE16BEC7BE1CC
:103C4000DFCF81E00E94241D812FDF91CF911F9152
:103C50000895539A2BB1277F3BB138604FB7F89442
:103C6000FC01CB01880F991F680F791F6E0F7F1F12
:103C7000E617F70789F0819198E03BB9000000C092
:103C800087FF2BB9880F000000C000C000C02BB90F
:103C900000C09A9591F7ECCF4FBF8FE594E0019764
:103CA000F1F700C0000008950895FC01680F791F26
:103CB0008FEF91E3E617F70771F02191822728E053
:103CC00030E087FF03C0880F892701C0880F21508B
:103CD0003109B9F7EFCF08950F931F93CF93DF9377
:103CE000C42FD22FFC0182818823C9F04093900217
:103CF0000E94202490938F0280938E0280E28C0F8A
:103D0000883008F057C0C77081E001C0880FCA959D
:103D1000EAF7DF91CF911F910F910C945F0580918D
:103D20009002481330C080918E0290918F020E94C1
:103D30003824883C910538F510E21D0FCD17B9F0F5
:103D400080E28C0F883040F4C77081E001C0880F9A
:103D5000CA95EAF70E946605183028F581E09D2F84
:103D6000977001C0880F9A95EAF70E945F05802F2F
:103D70000E9456051830F0F4D77081E001C0880F1A
:103D8000DA95EAF70AC080E28C0F883098F4C770A1
:103D900081E001C0880FCA95EAF7DF91CF911F91AA
:103DA0000F910C946605802FDF91CF911F910F9199
:103DB0000C945605DF91CF911F910F9108950F93A9
:103DC0009C01CB01243F4CE5340731F188F4293DB7
:103DD000FCE53F07D9F02A3D4CE5340779F1283D51
:103DE0003C45A9F506E221EE41EE68ED7CE52BC0ED
:103DF000263FFCE53F07E1F0A8F0273F3C4539F5B9
:103E000007E225EE46EE67EF7CE51DC007E225EEF2
:103E100045EE69ED7CE517C006E221EE40EE64EF69
:103E20007CE511C007E225EE44EE65EF7CE50BC0B2
:103E300006E221EE42EE66EF7CE505C008E221E0F5
:103E400045EE6AED7CE50E946C1E80E008C0FC0136
:103E50008281882319F01092900201C081E00F91B5
:103E60000895CF93DF93EC01FB018281882309F44D
:103E70001FC1C230FCE5DF0708F41BC1C6319CE559
:103E8000D90738F09E012B5F3C452930310508F0F9
:103E900010C10E94A20E9093A8028093A702C03185
:103EA000ECE5DE0709F4C3C008F041C0C8308CE57A
:103EB000D80709F49AC0F0F4C430ECE5DE0709F441
:103EC00087C068F4C2308CE5D80709F477C0C330E6
:103ED000DC4509F0E3C08091A702826076C0C6305D
:103EE000ECE5DE0709F46EC008F07BC08091A70204
:103EF00088606BC0CC308CE5D80709F485C068F4C5
:103F0000CA30ECE5DE0709F474C008F079C00E94FD
:103F1000EC078091A702806858C0CE308CE5D807A6
:103F200009F476C008F07FC08091A7028BC0CC3F17
:103F3000ECE5DE0709F44FC018F5C3318CE5D8076E
:103F400009F47DC078F4C131ECE5DE0709F473C0F3
:103F5000C231DC4509F0A2C00E94EC078091A702A3
:103F60008F7733C0C5318CE5D80709F472C008F4E7
:103F700086C0CB3FDC4509F091C08091A8023EC0CD
:103F8000C115FDE5DF0709F45FC058F4CE3F9CE59D
:103F9000D90709F444C008F43FC08091A8028260A8
:103FA0002DC0C230FDE5DF0709F475C008F45DC01F
:103FB000C330DD4509F072C080E06EC08091A70279
:103FC000816003C08091A70280618093A70266C0D0
:103FD0008091A70211C08091A80282608093A802FC
:103FE0005DC08091A7028062F0CF8091A7028064BB
:103FF000ECCF8091A70288608460E7CF8160EECF2C
:104000008091A7028E7FE1CF8091A7028D7FDDCFC7
:104010008091A702877FD9CF8091A80218C0809194
:10402000A8028D7FDBCF8091A7028F7ECECF8091BB
:10403000A7028F7DCACF8091A7028F7BC6CF8091C8
:10404000A702877F8B7FC1CF8091A8028D7F8E7F53
:10405000C5CF8091A70282FB222720F991E0922709
:1040600090FB82F990FB83F9B0CF8091A802982F42
:10407000909591708E7F892B90FB81F9AFCF0E9434
:10408000EC078091A70287FB222720F991E0922775
:1040900090FB87F99ACF81E00E94390F8091A702A7
:1040A0009091A8020E94B30E0E94EC0780E001C02C
:1040B00081E0DF91CF910895CF93DF9386319C45C6
:1040C00041F5EB010E94D00D982F8A8120910001CB
:1040D00030910101882379F09A7A81E009F480E037
:1040E00080939102911102C069E201C065E3C901A8
:1040F0000E944C230AC080919102811102C069E2A2
:1041000001C065E3C9010E944E230E94220E80E097
:1041100001C081E0DF91CF9108958EE1489B02C0FC
:104120008150E1F7489BFECF0895589880E28A9528
:10413000F1F7589A0895FC012AE02A95F1F728E052
:1041400090E080E031E040E14A95F1F7880F489B2C
:1041500002C08160932700C0000040E14A95F1F75A
:10416000215089F720E12A95F1F729B100C000001C
:1041700030E13A95F1F7217092272081920F9083D8
:104180000895EF92FF920F931F93CF93DF931F92A7
:10419000CDB7DEB719828C017C01E60EF11C0E153D
:1041A0001F0551F00E948D20CE0101960E949B2098
:1041B000F80181938F01F3CF81E09981911180E023
:1041C0000F90DF91CF911F910F91FF90EF90089585
:1041D000509A589A08955098589AE89AE9E6F0E06B
:1041E00080818C7F80830895615091E001C0990F98
:1041F0006A95EAF720E031E0992361F0492F4823DE
:1042000019F0589A232701C0589840E24A95F1F7CF
:104210009695F2CF222311F0589A01C0589880E267
:104220008A95F1F758980895FF920F931F93CF93B3
:10423000DF93EC018C01060F111DC017D10741F06F
:10424000F9900E94952068E08F2D0E94F420F5CF10
:10425000DF91CF911F910F91FF9008951F920F92C0
:104260000FB60F921124EF92FF920F931F932F938B
:104270003F934F935F936F937F938F939F93AF93EE
:10428000BF93EF93FF93CF93DF931F92CDB7DEB72A
:1042900019820E948D20CE0101960E949B20A82F9A
:1042A000A695A695A6959A2F969595702A2F257076
:1042B000920F292F237096959695920F87708913E8
:1042C0007CC08981811179C0A53008F076C080E179
:1042D0008A95F1F7589A509AB2E0BA95F1F700C072
:1042E0005898EA2EF12CEAE0AE9FD0011124AD5F80
:1042F000BE4F1896ED91FC9119973097B1F06091EF
:10430000B6017091B70116962D913C911797260F23
:10431000371F13968D919C911497680F791F1596EE
:104320004C91159712968C9109958AE08E9DF0011B
:104330008F9DF00D1124ED5FFE4F6581662351F0D6
:104340008091B6019091B70126813781820F931F2A
:104350000E9414210E949520F0E1FA95F1F75898F7
:104360005098589A80E18A95F1F78AE08E9D8001F5
:104370008F9D100D11240D5F1E4FD80112966C9168
:104380001297662399F08091B6019091B701139628
:104390002D913C911497820F931F0E94C120D80148
:1043A000ED91FC91811105C082E004C0D801ED912E
:1043B000FC9188E080830E948D200F90DF91CF9147
:1043C000FF91EF91BF91AF919F918F917F916F91ED
:1043D0005F914F913F912F911F910F91FF90EF901F
:1043E0000F900FBE0F901F9018950F931F93CF93B0
:1043F000DF93853091050CF0A9C02AE0289FF001D9
:10440000299FF00D1124ED5FFE4F20813181232B78
:1044100009F49CC0EC01F894509A589885E08A956C
:10442000F1F700008C2F869585709C2F9570890F71
:10443000982F9370869586958E0123E0000F111FAB
:104440002A95E1F7890F082B0E949520A4E0AA95F0
:10445000F1F700C068E0802F0E94F420B0E1BA9527
:10446000F1F75098589A489902C000C0FCCF87E0F5
:1044700090E0489B17C0019799F4509A589A8AE0A7
:104480008C9FF0018D9FF00D1124ED5FFE4F019088
:10449000F081E02D81E08083789481E090E058C045
:1044A00000C0E7CF8AE08C9F80018D9F100D112402
:1044B0000D5F1E4FF80165816623B9F08091B6014A
:1044C0009091B70126813781820F931F0E94C120EE
:1044D00081110BC0509A589AD801ED91FC9182E05D
:1044E0008083789482E090E033C00E948D20B0E217
:1044F000BA95F1F75898509AE0E1EA95F1F78AE019
:104500008C9FF0018D9FF00D1124ED5FFE4F6281B5
:10451000662351F08091B6019091B70123813481D7
:10452000820F931F0E9414210E9495208AE08C9F85
:10453000F0018D9FF00D1124ED5FFE4F0190F08191
:10454000E02D1082789480E090E002C084E090E05A
:10455000DF91CF911F910F910895909398028093CE
:10456000970208950E941E14811103C08091920247
:104570000895E0919702F0919802309721F0019010
:10458000F081E02D099480E00895E0919702F09188
:104590009802309721F00280F381E02D099408956C
:1045A000E0919702F0919802309739F022E0DC0117
:1045B0002C930480F581E02D0994089520919502B3
:1045C000309196022817390771F0909396028093E4
:1045D0009502E0919702F0919802309721F00680C1
:1045E000F781E02D0994089520919302309194026F
:1045F0002817390771F09093940280939302E09109
:104600009702F0919802309721F00084F185E02D17
:1046100009940895FC01329697E080E0915029F0CA
:1046200021912223D9F38F5FF9CF0895662349F0B2
:10463000FC01329608962191621729F0E817F907D4
:10464000D1F780E0089581E008959C01FC01329645
:104650009FEF80E04191461789F09F3F19F4411187
:1046600001C0982F8F5F8630A9F79F3F39F0F9017D
:10467000E90FF11D97FDFA956283089508959C0155
:104680002A5F3F4FFC014281461301C0128201960E
:1046900082179307B9F708950C9425230C943F23B0
:1046A000029626E0FC0111922A95E9F708951092EE
:1046B000EF021092F0021092F1021092F2020895AD
:1046C000CF92DF92EF92FF926B017C010E941E1449
:1046D00081110EC00E942C24C61AD70AE80AF90AD2
:1046E000C092EF02D092F002E092F102F092F20258
:1046F000FF90EF90DF90CF9008950F931F930E944B
:104700001E14882321F01F910F910C942C240E94D9
:104710002C240091EF021091F0022091F1023091CF
:10472000F202600F711F821F931F1F910F91089556
:10473000089508950C9499230C949923CF930E9483
:104740009C230E9493130E949A23C0E08C2F0E9406
:104750005D12811104C0CF5FCA30C1F701C081E092
:10476000CF9108950C9499230C94B2238091FB026D
:10477000843049F10E94B42380E00E94CF0310925C
:10478000990220E488E190E00FB6F894A895809310
:1047900060000FBE2093600083B7817F846083BF79
:1047A00083B7816083BF7894889583B78E7F83BFFA
:1047B0000FB6F894A895809160008861809360009E
:1047C000109260000FBE08950C9499230E94EC078C
:1047D0000E94B2220E94CF030C94E4231F920F92F6
:1047E0000FB60F9211248F939F93AF93BF93809135
:1047F0009902811113C08091F3029091F402A0916B
:10480000F502B091F6024196A11DB11D8093F3020D
:104810009093F402A093F502B093F602BF91AF918A
:104820009F918F910F900FBE0F901F90189582E06F
:1048300084BD93E095BD9AEF97BD80936E00089577
:104840002FB7F8948091F3029091F402A091F502B1
:10485000B091F6022FBF08952FB7F8946091F3023C
:104860007091F4028091F5029091F6022FBF0895A5
:104870009C014FB7F8948091F3029091F402A091BB
:10488000F502B091F6024FBF821B930B0895CF92B1
:10489000DF92EF92FF922FB7F894C090F302D0907E
:1048A000F402E090F502F090F6022FBFA701960106
:1048B000261B370B480B590BCA01B901FF90EF902B
:1048C000DF90CF90089578941F920F920FB60F92B9
:1048D00011248F939F93AF93BF938091F302909194
:1048E000F402A091F502B091F6020196A11DB11D4E
:1048F0008093F3029093F402A093F502B093F60232
:10490000BF91AF919F918F910F900FBE0F901F900D
:10491000189587E797E790930108809300089AE03D
:1049200088E10FB6F894A895809360000FBE90932D
:104930006000FFCF9093BB018093BA0108958091EE
:10494000A50208959091FB02943031F580939A026C
:1049500070939C0260939B0282E08093E9008FEF4A
:104960009091E800815095FD06C095ED9A95F1F77C
:1049700000008111F5CF8091E80085FF0DC040E077
:1049800050E063E070E08AE992E00E94B2268091F4
:10499000E8008E778093E8000895BC0184E00C94D1
:1049A000A224BC0183E00C94A22422E02093E9001D
:1049B0002FEF3091E800215035FD06C035ED3A95D6
:1049C000F1F700002111F5CF2091E80025FF0BC081
:1049D00040E050E066E070E00E94B2268091E8007E
:1049E0008E778093E8000895CF93DF9321E02093A2
:1049F000E9002FEF3091E800215035FD06C035ED7C
:104A00003A95F1F700002111F5CF2091E80025FF3C
:104A100014C0EC0140E050E068E070E00E94B22673
:104A20008091E8008E778093E80088E0FE01ADE990
:104A3000B2E001900D928A95E1F7DF91CF91089550
:104A40008091FA02811109C00E9443280E94A02887
:104A50008091E20084608093E20008951092FA024F
:104A6000089508950895089542E061EC81E00E9460
:104A7000BC2742E261EC82E00C94BC278091FD02ED
:104A8000833009F460C030F4813071F0823009F471
:104A900099C008958A3009F485C08B3009F46BC041
:104AA000893009F0A7C020C08091FC02813A09F04A
:104AB000A1C08091E800877F8093E8008091000387
:104AC00090910103892B21F468E08DE992E003C005
:104AD00060E080E090E070E00E94FD268091E800B8
:104AE0008B778093E80008958091FC02813209F071
:104AF00081C08091000390910103029708F07AC071
:104B00008091E800877F8093E8008091E80082FD33
:104B100005C08091FB028111F8CF6CC02091F30099
:104B20008091F20090E0922B029729F48091F1009D
:104B30008B7F813021F48091F1008093A5028091D8
:104B4000E8008B7753C08091FC02813A09F052C093
:104B50008091000390910103892B09F04BC0809153
:104B6000E800877F8093E8008091E80080FFFCCF19
:104B70008091420136C08091FC028132D9F580914A
:104B8000000390910103892BA9F58091E800877FAC
:104B90008093E8000E94F1278091FE0280934201F9
:104BA0000C94EC078091FC02813221F58091E800A1
:104BB000877F8093E8000E94F1278091FF02809315
:104BC000A60208958091FC02813AA1F48091E80048
:104BD000877F8093E8008091E80080FFFCCF809180
:104BE000A6028093F1008091E8008E778093E80020
:104BF0000C94F127089584B7877F84BF0FB6F8948B
:104C0000A895809160008861809360001092600098
:104C10000FBE90E080E80FB6F89480936100909307
:104C200061000FBE0C94670F0E9443280E94A028C9
:104C3000E2EEF0E080818460808378940E94352BDE
:104C40000E94750F88E391E00C94AD228091FB02E5
:104C50008530A9F48091FB02853079F40E94B62357
:104C60008091F9028823B1F30E949E23882391F357
:104C70000E949C260E94EC07EDCF0E94E6230C9434
:104C8000810F0C944326292F332723303105C9F097
:104C900060F42130310581F02230310509F044C043
:104CA0008BE390E02EE634E043C021323105E1F0A1
:104CB0002232310549F138C082E190E029EA34E03E
:104CC00037C099278130910549F028F0029761F5A6
:104CD000ECE2F4E005C0EAE6F4E002C0E4E5F4E06A
:104CE000849190E09F0124C06115710541F061300D
:104CF0007105D1F489E090E029E934E019C089E038
:104D000090E020E834E014C06115710541F0613095
:104D1000710551F48BE790E02BEB34E009C080E49F
:104D200090E026E335E004C080E090E020E030E051
:104D3000FA0131832083089580E189BD82E189BD34
:104D400009B400FEFDCF8091D8008F7D8093D800FC
:104D50008091E00082608093E0008091E00081FD1E
:104D6000FCCF0895CF92DF92EF92FF920F931F93A3
:104D7000CF93DF93EC018B017A010E9410288111FF
:104D800033C0E114F10439F0F70180819181081BEF
:104D9000190BC80FD91FC12CD12C0115110519F100
:104DA0008091E80085FD16C08091E8008E778093A1
:104DB000E800E114F10449F0F70180819181C80E07
:104DC000D91ED182C08285E00FC00E94102888239E
:104DD00021F30AC089918093F10001501109FFEF7E
:104DE000CF1ADF0ADACF80E0DF91CF911F910F91C8
:104DF000FF90EF90DF90CF900895209102033091C3
:104E000003032617370748F06115710539F420911F
:104E1000E8002E772093E80001C0B901FC0120E0F2
:104E20006115710579F18091FB028823F1F18530DC
:104E3000F1F18091E80083FD3CC08091E80082FDA3
:104E40002EC08091E80080FFEBCF2091F30080918D
:104E5000F20090E0922B6115710551F088309105B8
:104E600038F421912093F100615071090196F3CF3C
:104E700021E0089709F020E08091E8008E77809388
:104E8000E800CECF2111CFCF0AC08091FB0288234A
:104E900061F0853061F08091E80083FD0AC0809167
:104EA000E80082FFF2CF80E0089582E0089583E079
:104EB000089581E00895209102033091030326179D
:104EC000370748F06115710539F42091E8002E7715
:104ED0002093E80001C0B901FC0120E061157105D3
:104EE00091F18091FB02882309F440C0853009F4D8
:104EF0003FC08091E80083FD3DC08091E80082FDC5
:104F00002FC08091E80080FFE9CF2091F3008091CD
:104F1000F20090E0922B6115710559F088309105EF
:104F200040F424912093F10031966150710901966B
:104F3000F2CF21E0089709F020E08091E8008E7719
:104F40008093E800CBCF2111CCCF0AC08091FB0227
:104F5000882361F0853061F08091E80083FD0AC00C
:104F60008091E80082FFF2CF80E0089582E008950A
:104F700083E0089581E00895982F973068F5909325
:104F8000E900981739F07091EC002091ED005091F4
:104F9000F00003C0242F762F50E021FD02C09F5F58
:104FA000ECCF3091EB003E7F3093EB003091ED0081
:104FB0003D7F3093ED003091EB0031603093EB009A
:104FC0007093EC002093ED005093F0002091EE00E0
:104FD00027FDE5CF80E008958F708093E90081E0A0
:104FE00008958091FC0287FF11C08091E80082FD46
:104FF00005C08091FB028111F8CF11C08091E800BB
:105000008B770BC08091FB02882349F08091E800E8
:1050100080FFF8CF8091E8008E778093E8000895B4
:105020002091E4003091E50095E64091EC00842F5A
:10503000817040FF23C08091E80080FD1DC08091F9
:10504000FB02882399F0853099F08091EB0085FD73
:1050500011C04091E4005091E5002417350729F371
:10506000915011F09A01E1CF84E0089582E0089513
:1050700083E0089581E0089580E008954091E8007C
:1050800042FFDDCF08950E94B1280E94B928E0EECA
:10509000F0E0808181608083E8EDF0E080818F77AF
:1050A000808319BCA7EDB0E08C918E7F8C938081BA
:1050B0008F7E80831092FA0208950F931F93CF93EF
:1050C000DF930E94B1280E94B928C8EDD0E0888102
:1050D0008F77888388818068888388818F7D8883A3
:1050E00019BC1092FB021092F7021092F902109272
:1050F000F80200EE10E0F80180818B7F80838881C8
:105100008160888342E060E080E00E94BC27E1EE9D
:10511000F0E080818E7F8083E2EEF0E0808181602C
:105120008083808188608083F80180818E7F808386
:10513000888180618883DF91CF911F910F910895BD
:10514000E8EDF0E080818F7E8083E7EDF0E0808104
:105150008160808384E082BF81E08093FA020C94B6
:105160005D28E8EDF0E080818E7F80831092E20080
:1051700008951092DA001092E10008951F920F92A4
:105180000FB60F9211242F933F934F935F936F931A
:105190007F938F939F93AF93BF93EF93FF938091F0
:1051A000E10082FF0BC08091E20082FF07C0809186
:1051B000E1008B7F8093E1000E94342B8091DA0024
:1051C00080FF1FC08091D80080FF1BC08091DA0053
:1051D0008E7F8093DA008091D90080FF0DC080E13E
:1051E00089BD82E189BD09B400FEFDCF81E08093D5
:1051F000FB020E94202505C019BC1092FB020E94F0
:105200002E258091E10080FF19C08091E20080FF8F
:1052100015C08091E2008E7F8093E2008091E200D1
:1052200080618093E2008091D80080628093D800F2
:1052300019BC85E08093FB020E9432258091E10039
:1052400084FF30C08091E20084FF2CC080E189BDE2
:1052500082E189BD09B400FEFDCF8091D8008F7D29
:105260008093D8008091E1008F7E8093E10080914F
:10527000E2008F7E8093E2008091E2008160809363
:10528000E2008091F702882311F084E007C080914A
:10529000E30087FD02C081E001C083E08093FB0250
:1052A0000E9433258091E10083FF29C08091E200B4
:1052B00083FF25C08091E100877F8093E10082E039
:1052C0008093FB021092F7028091E1008E7F809321
:1052D000E1008091E2008E7F8093E2008091E20005
:1052E00080618093E20042E060E080E00E94BC27A1
:1052F0008091F00088608093F0000E943125FF913A
:10530000EF91BF91AF919F918F917F916F915F913D
:105310004F913F912F910F900FBE0F901F901895B6
:105320001F920F920FB60F9211242F933F934F931A
:105330005F936F937F938F939F93AF93BF93CF931D
:10534000DF93EF93FF93C091E900CF708091EC0061
:10535000D82FD17080FDD0E81092E9008091F00044
:10536000877F8093F00078940E94D4291092E900FE
:105370008091F00088608093F000CD2BCF70C093B7
:10538000E900FF91EF91DF91CF91BF91AF919F9194
:105390008F917F916F915F914F913F912F910F90DE
:1053A0000FBE0F901F9018951F93CF93DF93CDB72B
:1053B000DEB7AA970FB6F894DEBF0FBECDBFECEFF5
:1053C000F2E08091F100819323E0E430F207C9F725
:1053D0000E943E258091E80083FF2EC18091FC024F
:1053E0009091FD02492F50E04A30510508F024C148
:1053F000FA01EC58FF4F0C948A2B803821F0823848
:1054000009F01AC108C08091F8029091F90299231D
:1054100089F082600FC0809100038F70873008F0A0
:105420000BC18093E9008091EB0085FB882780F910
:105430001092E9009091E800977F9093E8008093A4
:10544000F1001092F100D1C0282F2D7F09F0F4C097
:10545000882319F0823061F0EFC08091FE02813024
:1054600009F0EAC0933009F080E08093F9022EC081
:105470008091FE0281112AC0809100038F702FEF6E
:10548000280F263008F0D8C08093E9002091EB0067
:1054900020FF1CC0933021F48091EB00806214C087
:1054A0009091EB0090619093EB0021E030E0A90136
:1054B00002C0440F551F8A95E2F74093EA0010920C
:1054C000EA008091EB0088608093EB001092E90085
:1054D0008091E800877F8093E8000E94F127ACC0AC
:1054E0008111AAC01091FE021F778091E30080789D
:1054F000812B8093E3008091E800877F8093E80010
:105500000E94F1278091E80080FFFCCF8091E300AA
:1055100080688093E300111102C082E001C083E043
:105520008093FB0289C08058823008F085C080914A
:10553000FE029091FF028C3D53E0950779F583E0E0
:105540008A838AE289834FB7F894DE01139620E0BC
:105550003EE051E2E32FF0E050935700E49120FF4A
:1055600003C0E295EF703F5FEF708E2F90E0EA305E
:1055700010F0C79601C0C0968D939D932F5F243184
:1055800049F74FBF8091E800877F8093E8006AE287
:1055900070E0CE0101960E94FD2616C060910003C6
:1055A00070910103AE014F5F5F4F0E944126BC0125
:1055B000892B09F441C09091E800977F9093E8000F
:1055C00089819A810E945B278091E8008B77809384
:1055D000E80032C0803881F58091E800877F8093B1
:1055E000E8008091F7028093F1008091E8008E77C7
:1055F00072CF811121C08091FE029091FF02992704
:105600000297D4F48091E800877F8093E80080912E
:10561000FE028093F7020E94F1278091F702811128
:1056200006C08091E30087FD02C081E001C084E0F4
:105630008093FB020E9434258091E80083FF0AC01A
:105640008091E800877F8093E8008091EB00806282
:105650008093EB00AA960FB6F894DEBF0FBECDBFC5
:10566000DF91CF911F9108950895CF938091FB0210
:105670008823A1F0C091E900CF709091EC00892FB0
:10568000817090FD80E8C82B1092E9008091E800BD
:1056900083FD0E94D429CF70C093E900CF91089573
:1056A0000E9443281092FB020895E8EDF0E080810B
:1056B000806180838AE18A95F1F700C08091D900EA
:1056C00081700895AA1BBB1B51E107C0AA1FBB1F15
:1056D000A617B70710F0A61BB70B881F991F5A957E
:1056E000A9F780959095BC01CD01089597FB072EF1
:1056F00016F4009407D077FD09D00E94622B07FCB6
:1057000005D03EF4909581959F4F089570956195D1
:105710007F4F0895EE0FFF1F0590F491E02D09943F
:10572000FB01DC0104C08D910190801921F44150EE
:105730005040C8F7881B990B0895FB01DC0102C09B
:1057400001900D9241505040D8F70895F999FECF3D
:1057500092BD81BDF89A992780B50895A6E1B0E081
:1057600044E050E00C94E02BA8E1B0E042E050E0CF
:105770000C94E02B262FF999FECF92BD81BDF89AAB
:10578000019700B4021639F01FBA20BD0FB6F89485
:10579000FA9AF99A0FBE08950396272F0E94BB2B01
:1057A0000E94BA2B252F0E94BB2B242F0C94BB2BBD
:1057B0000196272F0E94BB2B0C94BA2BDC01CB0146
:1057C000FC01F999FECF06C0F2BDE1BDF89A319611
:1057D00000B40D9241505040B8F70895F894FFCFAF
:1057E0002C0201BF020000000100000000BF020007
:1057F00000000501000000BF0204060000000000D8
:1058000000BF02080A0000000000002808641E14FF
:105810000A321E000E000E0E9F24F424D524D1243B
:10582000CD2401E200E900EA00B500B600B700CDE2
:10583000008301CC008A01920194012102230224F9
:10584000022502260227022A02B300B4006F00706C
:1058500000818283E200E900EA00B500B600B700EB
:10586000CD008301CC008A01920194012102230220
:1058700024022502260227022A02B300B4006F0088
:105880007000818283F5F6F7313332369497C6344F
:0A5890003500000000005202000184
:00000001FF
